:020000040000FA
:1000000048240020150200001D0200001F0200000D
:100010002102000023020000250200000000000071
:1000200000000000000000000000000027020000A7
:1000300029020000000000002B0200002D02000039
:100040002F020000A5020000A10500002F02000001
:100050002F0200002F0200002F0200002F020000DC
:100060002F0200002F0200002F0200002F020000CC
:100070002F0200002F0200002F0200002F020000BC
:100080002F0200002F0200002F0200002F020000AC
:10009000010300002F0200002F0200002F020000C9
:1000A0002F0200002F0200002F0200002F0200008C
:1000B0002F0200002F0200000000000000000000DE
:1000C0002F0200002F0200002F0200002F0200006C
:1000D0002F0200002F0200002F0200002F0200005C
:1000E0002F0200002F0200002F020000000000007D
:1000F000000000002F020000000000002F0200009E
:1001000000000000000000000000000000000000EF
:1001100000000000000000000000000000000000DF
:1001200000000000000000000000000000000000CF
:1001300000000000000000000000000000000000BF
:1001400000000000000000000000000000000000AF
:10015000000000000000000000000000000000009F
:10016000000000000000000000000000000000008F
:10017000000000000000000000000000000000007F
:10018000000000000000000000000000000000006F
:10019000000000000000000000000000000000005F
:1001A000000000000000000000000000000000004F
:1001B000000000000000000000000000000000003F
:1001C000000000000000000000000000000000002F
:1001D000000000000000000000000000000000001F
:1001E000000000000000000000000000000000000F
:1001F00000000000000000000000000000000000FF
:10020000DFF80CD000F03CF80048004789080000F7
:10021000482400200648804706480047FEE7FEE7DE
:10022000FEE7FEE7FEE7FEE7FEE7FEE7FEE7FEE7A6
:10023000590300000102000040EA01039B0703D0BC
:1002400009E008C9121F08C0042AFAD203E011F815
:10025000013B00F8013B521EF9D27047D2B201E0D7
:1002600000F8012B491EFBD270470022F6E710B5BB
:1002700013460A4604461946FFF7F0FF204610BD14
:10028000064C074D06E0E06840F0010394E80700E3
:1002900098471034AC42F6D3FFF7B6FFB81300000E
:1002A000D813000070B5144CD4F80001002628B112
:1002B000D4F80403C00701D0C4F80061D4F80C01DD
:1002C0000E4D40B1D4F80403000704D5C4F80C6106
:1002D000286900B18047D4F8100100280BD0D4F869
:1002E0000403C00607D5C4F81061E868002802D0EE
:1002F000BDE87040004770BD001000403000002095
:100300007CB5144C606A01902078002821D001202F
:1003100000F059F9656800266660012000F064F974
:10032000E169002915D0E80703D08DF80060684620
:100330008847A80705D501208DF80000E1696846C7
:100340008847680705D502208DF80000E1696846F6
:1003500088477CBD30000020F0B54FF080527F4EC2
:10036000D2F830017E4FD2F83411431C08D0054634
:100370004FEA010400234FF0010C082D05D013E0D3
:100380003B783578C3F30314F4E72CB1012C03D088
:10039000022C01D0032C07D14FF08044C4F80C315B
:1003A000C4F810316F4C2360441C04D005460C4641
:1003B000082D05D061E03C783578C4F30314F7E7E5
:1003C0002CB1012C03D0022C01D0032C55D1664C4A
:1003D0002468664D2C60644C241D24682D1D2C60FF
:1003E000614C083424682D1D2C605F4C0C3424684B
:1003F0002D1D2C605C4C103424682D1D2C605A4C33
:10040000143424682D1D2C60574C18342468574D23
:1004100020352C60544C1C3424682D1D2C60524C0B
:10042000203424682D1D2C604F4C243424682D1D4D
:100430002C604D4C283424682D1D2C604A4C2C34E3
:1004400024682D1D2C60484C30342468474D4035BD
:100450002C60454C343424682D1D2C60424C3834BB
:1004600024682D1D2C60404C3C3424682D1D2C60CC
:100470003D4C403424682D1D2C60082804D10C000C
:1004800002D13C4D3A4C2C60082804D10C0002D11A
:10049000394DFB242C60082808D10C0006D192F8B5
:1004A0005852364A146865F303041460082804D1CE
:1004B0000A0002D1324C82012260421C03D13978F9
:1004C0003078C1F3031108280DD129B1012903D0D7
:1004D000022901D0032906D12A480168C90702D0A0
:1004E0006FF0010101602848016841F4700101606A
:1004F000BFF34F8FBFF36F8F4FF01021D1F8000281
:10050000002803DBD1F80402002823DA1F4AC2F8CE
:1005100000C01F480468002CFCD01224C1F800421F
:100520000568002DFCD0C1F8044201680029FCD008
:10053000136001680029FCD0BFF34F8F12487C384C
:100540000168144A01F4E06111430160BFF34F8F69
:1005500000BFFDE7114910480860F0BDE00F00F052
:10056000E80F00F0380500400404001020C50040EA
:10057000488103008C56004018F50040E40E00400E
:10058000409602400004004088ED00E004E5014090
:1005900000E401400400FA050090D0037800002038
:1005A000014800680047000028000020002809DBFF
:1005B00000F01F02012191404009800000F1E0207D
:1005C000C0F88012704700280DDB00F01F020121E7
:1005D00091404009800000F1E020C0F88011BFF395
:1005E0004F8FBFF36F8F7047002809DB00F01F02A9
:1005F000012191404009800000F1E020C0F8001185
:100600007047002809DB00F01F02012191404009DA
:10061000800000F1E020C0F8001270474907090E81
:10062000002804DB00F1E02080F80014704700F09F
:100630000F0000F1E02080F8141D704702E008C8A8
:10064000121F08C1002AFAD170477047002001E04C
:1006500001C1121F002AFBD17047006890FAA0F078
:1006600000BA00BA7047000072B609480068C007B7
:1006700000D000BEBFF34F8F0548E4380168054A3B
:1006800001F4E06111430160BFF34F8F00BFFDE74C
:10069000F0ED00E00400FA050EB500210091CDE96F
:1006A00001106A4644F20100FFF7DEFF0EBD0000B4
:1006B0002DE9FC410646C0074FF000050ED0104F53
:1006C00000240122385D009500231146019500F0B9
:1006D0005DFB641C042CF4D300F01CF8B0070DD5AE
:1006E000074E0024361D0022305D0323009511467D
:1006F000019500F04BFB641C042CF4D3BDE8FC8195
:10070000B01300000249085C012100F088BB000022
:10071000B013000010B500242046FFF7F3FF641C5F
:10072000042CF9D310BD006890FAA0F000BA70470D
:100730004FF080400021C0F800110121C0F80010E6
:10074000D0F800110029FBD07047000000B51BA0B5
:100750008BB0006808901AA01AA100680990D1E92E
:100760000001CDE90601182218496846FFF764FD2B
:1007700001208DF800008DF8080015480190002038
:100780008DF801004FF416718DF81400ADF80C10BF
:10079000684600F01BF900280DD108A800F0E0F928
:1007A000002808D109A800F0EDF9002803D108219C
:1007B00006A800F0F9F90BB000BD0000E7E7E7E795
:1007C000C2C2C2C2E7C2C3C4C5C6C7C8981300002C
:1007D00071090000F8B508240F2503266846009427
:1007E00000F0EEFA009900EB8100C0F80067641C8D
:1007F000AC42F3D9BDE8F8400120FFF759BF000033
:1008000070B500F017FC1E490020A1F5947300BFDD
:1008100000EB800202EB40121A4441F82020401CF9
:100820000828F5DB164900202C3101F5947200BF31
:1008300000EB800404EB40140C4442F82040401CC0
:100840000828F5DB00200F4A4FEA000100EB800486
:1008500004EB4014E51800EB4004401C42F824501F
:1008600002EB840408282171A160EFDB054A002017
:1008700012F1600242F82010401C0828FADB70BD1B
:10088000E4010020A8030020FFF7A4FFFFF750FFBA
:10089000FFF75CFF08B1FFF7FFFE214C214D224E10
:1008A0000027E7701E4800F0D9F9A0BBA0794107E6
:1008B00003D000F00700042801D9012100E0002145
:1008C0000D2000F099FAA07900F00700012801D965
:1008D000052801D9012100E000210E2000F08CFA4A
:1008E000A07900F00700022801D9062801D90121CA
:1008F00000E000210F2000F07FFAA07900F007004F
:10090000032801D8012100E00021102000F074FA32
:10091000A079401CA071691C30468847C1E70000DF
:10092000000000209013000000D4300070B50C4986
:100930004FF4705008600B4C00256570257000F076
:1009400079FB20210848FFF790FCE562142025631D
:10095000FFF739FE05490320C1F80002002070BDF1
:1009600008F501403000002028040020001000405D
:1009700010B50078002808D0012807D0022804D13B
:10098000054800F0A9F80028FAD010BD00F006F8DC
:10099000BDE8104000F04EB97C000020094810B5B9
:1009A000007860B10120FFF70EFE07480021816248
:1009B000016241620120FFF717FE002010BD0820F0
:1009C00010BD000030000020E401002070B50500DB
:1009D00065D0354C207818B1FFF7A8FF00285DD10D
:1009E0006868E061182229463048FFF725FC002599
:1009F000656020212E48FFF738FCE562256300F092
:100A000049FCE8B32B494FF0E7300860091D4FF06F
:100A100043300860091D28480860091D2748086000
:100A2000FFF7EEFE264904200860254808380560D7
:100A3000244840F20221C0F80012244A22491160E1
:100A4000111D08602048001D091D08601D48103058
:100A5000091D0860091D1E4808601B48F038091D63
:100A600008601B48001D091D0860091D1948086021
:100A70000E4E707C00F007010120FFF7CFFD00E073
:100A80000FE0B07C00F007011420FFF7C7FD142031
:100A9000FFF7AAFD657001202070002070BD0E20B8
:100AA00070BD072070BD000030000020A4000020B1
:100AB000280400201C150040E743C323A363E3136D
:100AC00010A5004000A000400011004060F501406A
:100AD00040A100400010004070B505461E48007857
:100AE00080B385B31D4CA06A70B30120FFF76BFD86
:100AF000606A54F820100A782A7054F82010497857
:100B0000697054F820108978A97054F82010097978
:100B1000297154F82010C978E97054F82010681D24
:100B2000491DFFF789FB606A401C6062082801D3F9
:100B300000206062A06A401EA0620120FFF754FD01
:100B4000002070BD01E002E003E00820F9E70E207C
:100B5000F7E70520F5E7000030000020380300200B
:100B6000074910B54A780AB1112010BD30B10068AC
:100B70004863012000F042FB002010BD0E2010BD94
:100B800030000020074910B54A780AB1112010BD85
:100B900030B100688863022000F030FB002010BDF7
:100BA0000E2010BD3000002010B50C460F494978CA
:100BB00009B1112010BD18B1082C03D9072010BDB0
:100BC0000E2010BD0146094822463C30FFF734FB99
:100BD0000648C4F108023430FF210474D140817406
:100BE000042000F00BFB002010BD000030000020AE
:100BF0000E4810B50078A0B10D4CA06A98B1012044
:100C0000FFF7E1FCA06A401EA062606A401C6062BF
:100C1000082801D3002060620120FFF7E5FC0020D6
:100C200010BD082010BD4FF4807010BD30000020B2
:100C3000E4010020074810B5407808B1112010BD2C
:100C40000548806A18B100F04FFA002010BD4FF43B
:100C5000807010BD30000020E40100202DE9F04735
:100C6000DFF818A106469AF8000040B156B1307876
:100C700068B120280BD8424F397829B109E0082003
:100C8000BDE8F0870E20FBE7F97C884201D90920F6
:100C9000F6E73C4CA06A082801D30420F0E77078FE
:100CA000082801D30720EBE70120FFF78CFCDFF8D1
:100CB000CC8078784FF0000908F12C0860B13249F7
:100CC000002000BF00EB400201EB82021279EAB182
:100CD000401C0828F6DB42E0206A2522314654F801
:100CE0002000FFF7A9FA727818F80210491C01F0E9
:100CF000030108F80210206A54F82020401C08283C
:100D00001171206228D3C4F8209025E000EB400048
:100D100011EB800523D001202871C5F80890252209
:100D200031462868FFF788FA727818F80210491CD3
:100D300001F0030108F802102868134A0171717864
:100D4000603252F8210018B942F8215004E00846F8
:100D500081680029FBD18560A06A401CA062012047
:100D6000FFF742FC787830B9387C20B99AF8010056
:100D700008B900F0B9F9002082E700003000002037
:100D8000A4000020E4010020A80300202DE9FF4179
:100D90001C46DDE90A7815460E46684600F01EF846
:100DA00046EA450141EA840141EA072242EA084154
:100DB000009A00EB8200C0F80017BDE8FF81000038
:100DC0000168202902D24FF0A040704701F01F01B6
:100DD00001600148704700000003005001682029AD
:100DE00002D24FF0A040704701F01F01016001489E
:100DF000704700000003005038B501240090684699
:100E000031B1FFF7DDFF00998C40C0F8084538BDCF
:100E1000FFF7D6FF00998C40C0F80C4538BD38B5B7
:100E200001240090684631B1FFF7D8FF00998C404B
:100E3000C0F8084538BDFFF7D1FF00998C40C0F8D5
:100E40000C4538BD70B5164CA068164AC2F80002B1
:100E5000A06A15490860154B091D988982380860F9
:100E60001348012140F80C1F0021C0F83411C0F8CC
:100E70003811104D4FF4E050286050142D1D28609B
:100E8000C2F80C11187810B96169002088470B4925
:100E9000094808600A48E0600320607070BD0000E7
:100EA000300000200010004040A50040A4000020B9
:100EB00000A0004004F50140860300200415004016
:100EC000010F000010B50C4C606840F0010060603C
:100ED000FFF78EFE0948806A30B11420FFF791FBBE
:100EE000BDE8104000F000B900206070BDE810407F
:100EF0001420FFF786BB000030000020E401002032
:100F00002DE9F047414A4FF4E05010604049D1F8D4
:100F10000C31DFF8009100273F4CB9F80E004E1459
:100F2000DFF8F8800125E3B33D4B1B68CBB32561A7
:100F30001660D8F8041041F00101C8F80410D8F880
:100F40002010401A401CC8F82400FFF751FE99F801
:100F5000000088B109F2E220017869B140784108C7
:100F600030480068C0B200F073F828B1D8F8040027
:100F700040F00400C8F804002B48806A50B199F88A
:100F80001000012806D01420FFF73BFBBDE8F04716
:100F900000F0AAB888F80170BDE8F0471420FFF708
:100FA00030BBD8F820C0BCF1010CC8F820C00BD26F
:100FB00025611660401CC8F82400D8F8040040F0F1
:100FC0000200C8F80400E5E7D8F808000F4640F032
:100FD0000802C1F80022D8F81800D8F814100078D8
:100FE000884710481149283801601148C8F80C009A
:100FF000022088F8010025600448001F0660D4F82C
:101000004401002800D03D60BDE8F08708F50140AC
:1010100000100040A400002000A00040300000208C
:10102000001400402C150040E4010020640300205F
:10103000450E00000549002008624862886201F5FB
:10104000AA7108624862886270470000E4010020CB
:101050002DE9F041224C07468846A06A08283DD277
:10106000A4F5257120460A780026006A01F2E225DF
:10107000012A03D04A7842B1C97C02E029782029AC
:101080002CD854F82020117002E054F820100E7073
:1010900054F82000A91C10F8052BFFF7CDF8206AA2
:1010A00054F820104F700F49096854F820209170AF
:1010B00054F8202082F80480697854F8202041F305
:1010C0000001491C401CD1702062082800D3266210
:1010D000A06A401CA0620120BDE8F0810020FBE76F
:1010E00038030020481500402DE9F05F3D4C4FF0DB
:1010F0000108C4F824803C48DFF8F0A0A0F5A077F0
:10110000416A3B4D4FF0000B50F82110A161387837
:1011100007F5307610B1012843D10DE008786169F8
:101120008847A1690879307086F801B011F8052B5D
:10113000B01CFFF781F818E0C87820B3387D10B3F1
:10114000002081460878307008794006000E7070E3
:10115000CA78D2B100221043707011F8052BB01C70
:10116000FFF76AF8B9F1000F11D0A06840F008004D
:10117000C5F800021120C5F80403F8892062022096
:10118000C4F80CA00CE00120DBE70122E3E7A06833
:10119000C5F800021020C5F804031648E060404678
:1011A0006070A069144A417811604078444608FA9A
:1011B00000F0111D08600B480F4934302439C07C01
:1011C0000860081F06600120FFF7F0F90120FFF713
:1011D0000BFAC5F804B1C5F808B1C5F810B12C6018
:1011E000BDE8F09F30000020E4010020450E000023
:1011F00000100040C50E00002C15004010B504463C
:10120000C00704D00F48FFF728FA0F490860A0076D
:1012100006D50C48001DFFF720FA0B49091D086090
:1012200060070DD507480830FFF77DFA06490831F9
:10123000086004480C30FFF776FA03490C31086067
:1012400010BD0000640000201C1500400E490F482E
:101250000A7A02600E48492352B1012A05D0032AB6
:1012600006D0042A01D0002070473022826200E0BC
:1012700083628B89826A3E32934202D2806A3E3018
:101280008881012070470000A40000201015004054
:101290003000002070B500F03FF8FFF7D7FF184985
:1012A000184A0B787BB1012B0BD000230340164862
:1012B0004D7A041FB5B1012D0ED0022D07D00024A8
:1012C00017E0124B00E0124B53610123EEE74FF69B
:1012D000FF7606600F4803E0FF26066040F2071025
:1012E000206002E000260660266007480838056096
:1012F0000124C87C51691C408847204670BD00000D
:10130000A4000020300000203C15004059130000CC
:101310002D1300002110010002480349807A086063
:1013200070470000A40000200C150040084A07493F
:1013300011600849497C491E090441EA0021014322
:1013400041F08070111D086070470000000101002D
:10135000141500406400002007490648086007484B
:101360000749407C401E41EA00400349091D0860CE
:1013700070470000060003001415004064000020C0
:10138000200000010000000000000000000000003C
:101390000338FDD870470000010000000000000085
:1013A00001020000FA00030000010220000000001A
:1013B0000D0E0F100B0C1819D813000000000020A0
:1013C0007C0000003C060000541400007C0000205B
:1013D000CC2300004C0600000800000000010000C3
:1013E00000110000000000000000000000000000EC
:1013F00000000000000000000000000000000000ED
:1014000000000000000000000000000000000000DC
:1014100013010000000000000000000000000000B8
:1014200000000000000000000000000000000000BC
:10143000000000000000000000000000E7E7E7E710
:10144000C2C2C2C2E7C2C3C4C5C6C7C80805FF023C
:041450000090D00335
:0400000500000201F4
:00000001FF
